:020000020000FC
:0200000003C03B
:100004001CC01BC00FED0DBF00E00ABB0FEF0BBB04
:1000140004E007BB03E008BB00E30BBF0FEF02BB28
:1000240003E000BD00E305BF00E808B90FE000B934
:100034006627772778948895FECF09B316B31C6F8B
:100044005FEF0517150729F46627772753E058BB98
:10005400189506171707B80111F018D0EECF01D084
:10006400ECCF22E08FD087D086D085D084D083D0C7
:1000740082D081D080D07FD07ED07DD07CD07BD008
:100084007AD079D078D02A9569F7089522E07AD089
:1000940011FD6AD011FF6FD075D010FD65D010FF2F
:1000A4006AD070D007FD60D007FF65D06BD006FD25
:1000B4005BD006FF60D066D005FD56D005FF5BD04F
:1000C40061D004FD51D004FF56D05CD003FD4CD068
:1000D40003FF51D057D002FD47D002FF4CD052D07D
:1000E40001FD42D001FF47D04DD000FD3DD000FFBF
:1000F40042D048D011FF38D011FD3DD043D010FF7D
:1001040033D010FD38D03ED007FF2ED007FD33D0BA
:1001140039D006FF29D006FD2ED034D005FF24D0D7
:1001240005FD29D02FD004FF1FD004FD24D02AD0F0
:1001340003FF1AD003FD1FD025D002FF15D002FD06
:100144001AD020D001FF10D001FD15D01BD000FF24
:100154000BD000FD10D016D00ED00DD00CD00BD08B
:100164002A9509F094CF089530E148E04A95F1F7D3
:100174003A95D9F7089530E448E04A95F1F73A956D
:10018400D9F7089530E157E058BB000042E04A95A2
:10019400F1F753E058BB000044E04A95F1F73A9573
:0401A40091F7089532
:00000001FF
